:100000008C019D018F019001910192019301940156
:1000100095019601980199019A0183161030850087
:1000200000308600640027308100831290289B01F5
:100030000C089C006D200314980203182A2803144E
:100040000130990203182A28031401309A02031878
:100050002A281B149C031C086D2003149902031802
:100060003728031401309A02031837281B149C0305
:100070001C086D2003149A02031840280314412819
:100080001B0C00349B010C089C006D20031098078A
:10009000031C5528031001309907031C5528031031
:1000A00001309A07031C55281B149C031C086D2063
:1000B00003109907031C6228031001309A07031CE0
:1000C00062281B149C031C086D2003149A07031C50
:1000D0006B2803146C281B0C003482070034003496
:1000E0000A3400340034643400340334E834003417
:1000F0002734103401348634A0340F344234403471
:1001000082073F3406345B344F3466346D347D34BB
:1001100007347F346734803482070D34BB34A03415
:10012000831600308600831211308C0009308D0058
:100130008E0106309D0017200318A5288E0A8D0316
:10014000031D9B2803308C02A828422003308C0218
:1001500009308D0010301D079B009B031B08840095
:100160000E088E0180009D0301300C07031D9B28A3
:1001700018088F0097018101000000009D013C30AC
:100180008C008B0110308500831618308500831297
:100190000F301D078400000880209B0005300315E8
:1001A0001D02031DD9289B1700000000000000005D
:1001B000DF28023003151D02031DDF289B171B08D3
:1001C00086001D08000085000B1DE928970A0B1109
:1001D000EC2800000000000005309B009B0BEE287F
:1001E000000000009D0A073003111D02031DC828EE
:1001F000000003309B009B0BFB2800000000000068
:100200009D018C0BC828000031309B009B0B0629F8
:10021000000000000B1D0F29970A0B111229000086
:1002200000000000030186001030850083161030A6
:10023000850083120B19970A0B1101089900170802
:100240009A009B019B0A851585110B11010803116A
:100250001902031922299B0A9B099B0A1B0A980071
:10026000173085008316013086008312061C392959
:10027000932900308C20031403111A02031C522905
:10028000031D622901308C20031103141902031C81
:100290005229031D622902308C2003141802031C0A
:1002A0005229622900308C208F001A0893000130F7
:1002B0008C2090001908940002308C2091001808BE
:1002C0009500712900308C2093001A088F000130AE
:1002D0008C2094001908900002308C20950018089A
:1002E00091001508031491020318802903140130AA
:1002F000900203188029031401308F02031880290B
:1003000014080314900203188A29031401308F0281
:1003100003188A2913088F020F089A001008990001
:1003200011089800B32902308C2003109807031C91
:10033000A429031001309907031CA42903100130DC
:100340009A07031CA4291B1401308C200310990761
:10035000031CB029031001309A07031CB0291B1499
:0C03600003018C209A07103085009028C3
:00000001FF
